:020000020000FC
:1000000004E00EBF0FE51FEF2FEF17D00DBF0FEF6E
:100010000ABB0FEF07BB00EC01BB00E002BB10E026
:1000200020E027D011E021E024D012E022E021D00E
:1000300013E023E01ED01FEF09D0012F1A95000016
:10004000E1F7102F2A950000C1F7089501E0412F34
:100050004023041729F04FE342BB4FEB42BB05C0DE
:100060004FE742BB4FEF42BB00C0000F003079F7B3
:100070000895022F0F70103039F0113051F0123006
:1000800069F01330A1F008954BB3407F402B4BBB78
:10009000089548B3407F402B48BB08954BB34F7041
:1000A000000F000F000F000F402B4BBB089548B30B
:1000B0004F70000F000F000F000F402B48BB08953A
:00000001FF
